:100000000C942A001895000018950000189500001F
:10001000189500001895000018950000189500002C
:10002000189500001895000018950000189500001C
:10003000189500001895000018950000189500000C
:1000400018950000189500001895000018950000FC
:10005000189500008FE58DBFC0E4E8E34E2E88E0E0
:100060008EBFD8E0F8E05F2EEEEFF7E0A0E6B0E05C
:10007000A89584B7082E877F84BF88E1992781BD22
:1000800091BD88278D933197E9F76624D29ADA9A41
:100090008EE190E00E946400DA98E2E0F0E00E94D5
:1000A00055000C944700F894FFCF88EE93E00CD0F5
:1000B0003197D9F708953197F1F70895689462F868
:1000C0000895E89462F80895EF93FF93EE27E82BE4
:1000D000E92B31F0E0EAFFE03197F1F70197D1F732
:0600E000FF91EF9108956D
:00000001FF
